:040000008A11E32F4F
:100B860064008001840A0406031900340406C42D97
:100B96007E088A007F088200CB258A118000840A9D
:100BA60004087D0603190034FF0A0319FE0ACF2D37
:100BB600EB2DF930F4006400F40BDE2DE22D640019
:100BC600FF3083120313CE070318CF0AFF30CF0777
:100BD600831203134F084E04031DF22DF32DDC2D53
:100BE600080083120313D00085140330F500F50BBB
:100BF600FA2D8312031385100030D1000030D20085
:100C0600003083120313D3000030D4008312031381
:100C160005150330F500F50B0E2E8312031305118F
:100C2600500853078A1109278A1186000230CE0020
:100C36000030CF008A11DB258A110130831203139D
:100C4600D3070318D40A0030D4075408803AF500B5
:100C560080307502031D312E05305302031C342EDD
:100C6600352E092E013083120313D1070318D20A39
:100C76000030D2075208803AF50080307502031D15
:100C8600462E64305102031C492E4A2E032E0800BC
:100C960098130730831603139C00031000300318C3
:100CA60001309D0003100030031801309B001830FE
:100CB6008500031000300318013086000310003051
:100CC6000318013083120313850003100030031844
:100CD6000130860001308A11F4258A1106308A1106
:100CE600F4258A110B308A11F4258A111F308A11D6
:100CF600F4258A1174308A11F4258A1129308A1153
:100D0600F4258A112E308A11F4258A1133308A117E
:100D1600F4258A1138308A11F4258A113D308A115A
:100D2600F4258A1142308A11F4258A1147308A1136
:100D3600F4258A114C308A11F4258A1151308A1112
:100D4600F4258A115B308A11F4258A1165308A11DF
:100D5600F4258A116A308A11F4258A116F308A11B6
:100D6600F4258A1179308A11F4258A1188308A117E
:100D7600F4258A1192308A11F4258A119C308A1141
:100D8600F4258A11A1308A11F4258A11A6308A1118
:100D9600F4258A11AB308A11F4258A11B0308A11F4
:100DA600F4258A1110308A11F4258A1197308A1198
:100DB600F4258A1124308A11F4258A118D308A117E
:100DC600F4258A111A308A11F4258A1115308A11F0
:100DD600F4258A117E308A11F4258A1183308A110E
:100DE600F4258A1160308A11F4258A1156308A1149
:100DF600F4258A116D2E8A110028FE00FE1F082F89
:100E060083137E188317000808000408FE000730C5
:100E16008A007E0882070034FC34123412341234FD
:100E2600FC34FE349234923492346C347C34823402
:100E36008234823444347C348234823482347C3446
:100E46005E3492349234923462341034183414344A
:100E5600FE341034FE348234823482347C3484345A
:100E6600C234A23492348C34FE3412341234123426
:100E760002347C349234923492347434FE34103416
:100E860010341034FE3400348234FE34823400349C
:100E960070348034803480347E34FE341034283408
:100EA60044348234FE348034803480348034FE34DA
:100EB600043418340434FE34FE3408341034203438
:100EC600FE344C349234923492347C347C34823402
:100ED600823482347C346C349234923492346C345E
:100EE600FE341234123412340C34FC348234A234FC
:100EF6004234BC34FE341234323452348C34FE3430
:100F060092349234923482344C3492349234923401
:100F160064347C349234923492346434823442346D
:100F2600223412340E3402340234FE3402340234D3
:100F360044348234923492346C347E348034803437
:100F460080347E3400348434FE34803400343E34BD
:100F56004034803440343E34FE34403430344034FF
:100F6600FE34C634283410342834C63406340834E3
:100F7600F03408340634C234A23492348A348634C7
:100F8600303431343234333434343534363437341F
:100F960038343934413442344334443445344634A5
:100FA600EE34ED34EB34E734DE34DD34DB34D73481
:100FB600BE34BD34BB34B7347E347D347B347734B1
:100FC600763084007C308A11C3258A118313403021
:100FD60084004E308A11C3258A114030FD00073047
:100FE600FE00C330FF00203084008A11CF258A110D
:060FF60083018A114B2E5D
:00000001FF
